:0400000069EF00F0B4
:0E0008002282FACF01F0FBCF02F06BED00F088
:100018002280D8CF0FF0E8CF10F0E0CF11F0FACF60
:1000280012F0FBCF13F0E9CF14F0EACF15F0E1CFCF
:1000380016F0E2CF17F0D9CF18F0DACF19F0F3CFD6
:100048001AF0F4CF1BF0F6CF1CF0F7CF1DF0F8CF65
:100058001EF0F5CF1FF0F2B4F2AA0AD0FA0ED65E5F
:10006800000ED75AF2940F0EC16ECF0E936E8A8A85
:100078009DB09EA006D09E90204A212A000E946E24
:100088008B8C1FC0F5FF1EC0F8FF1DC0F7FF1CC0FA
:10009800F6FF1BC0F4FF1AC0F3FF19C0DAFF18C03F
:1000A800D9FF17C0E2FF16C0E1FF15C0EAFF14C070
:1000B800E9FF13C0FBFF12C0FAFF11C0E0FF10C038
:1000C800E8FF0FC0D8FF22901000B9EF00F006003B
:1000D800E9CF03F0EACF04F0E1CF05F0E2CF06F074
:1000E800D9CF07F0DACF08F0F3CF09F0F4CF0AF050
:1000F800F6CF0BF0F7CF0CF0F8CF0DF0F5CF0EF0F0
:100108009DB09EA006D09E90204A212A010E946E92
:100118008B8E0EC0F5FF0DC0F8FF0CC0F7FF0BC0AB
:10012800F6FF0AC0F4FF09C0F3FF08C0DAFF07C0F2
:10013800D9FF06C0E2FF05C0E1FF04C0EAFF03C023
:10014800E9FF02C0FBFF01C0FAFF22921100010E75
:10015800CD6E9D80F28CD08E9F80F28E9E90000E88
:10016800D56EF28AF194D58EFFD7216A206A229043
:0801780022920001ABEF00F040
:020000040020DA
:08000000FFFFFFFFFFFFFFFF00
:020000040030CA
:0E00000000051F1FFF8385FF0FC00FE00F409C
:00000001FF
